:100000000C941E060C9473280C94A0280C9446069D
:100010000C9446060C9446060C9446060C94460630
:100020000C9446060C9446060C9432130C94460627
:100030000C9446060C9446060C9446060C94460610
:100040000C94CD280C9446060C94BB2C0C94FE2CDE
:100050000C9446060C9446060C9446060C944606F0
:100060000C9446060C944606E118431922192519EA
:1000700028192B192E193119341943193D19751ADC
:10008000771A771A751A771A771A771A771A771AEA
:10009000771A771A771A771A771A771A771A771AD8
:1000A000FB19771A771A771A771A771A6C19771A51
:1000B000771A771A771A771A771A771A771A771AB8
:1000C000771A771A771A771A771A771A071A071A88
:1000D000071A071A071A071A071A071A071A771AA8
:1000E000771A771A771A771A771A6C19061A061A76
:1000F000061A061A771A141A1A1A201A261A2C1A0D
:10010000321A381A3E1A481A521A5C1A661AAD196F
:100110006F19771A771A771A771AFB19771A771ADD
:10012000771A771A771A771A771A771A051A051A2B
:10013000051A051A771A141A1A1A201A261A2C1ACE
:10014000321A381A3E1A481A521A5C1A661AAD192F
:100150006F19771A771A771A771AFB19AA1AAA1A37
:10016000AA1AAA1AAA1AAA1AAA1AAA1AAA1AAA1A6F
:10017000AA1AAA1AAA1AC01BC01BC01BC01BC01BEC
:10018000C01BEF1AF91A031B0D1B6A1B741B831B80
:10019000941B1C1D311D3D1D461D551D7A1D831DC3
:1001A000CC1D951DE120E720ED20F4200221242123
:1001B0004221456E746572206D656E752E2E2E007F
:1001C000546F67676C6564206D6963726F50504D42
:1001D00000546F67676C656420696E76657274653C
:1001E000642050504D2100546F67676C6564205443
:1001F00058206D7574696E672100546F67676C6570
:10020000642074656C656D65747279210050726F3D
:10021000746F636F6C206572726F72207769746897
:100220002052580054696D656F7574207768656E4B
:1002300020636F6E6E656374696E6720746F205201
:100240005800507265737320616E79206B65792058
:10025000746F2063616E63656C00436F6E6E6563DF
:1002600074696E6720746F2052582C20706F776508
:100270007220757020746865205258202877697440
:10028000682062696E6420706C7567206966206EF4
:100290006F74207573696E6720616C776179732064
:1002A00062696E642900546F67676C656420276912
:1002B0006D6D656469617465206F75747075742700
:1002C00000546F67676C65642027736C61766520E6
:1002D0006D6F64652700546F67676C6564202761E4
:1002E0006C776179732062696E642700546F676769
:1002F0006C65642050504D206368616E6E656C20A3
:100300006C696D69740053657420525353492069B8
:100310006E6A656374696F6E206368616E6E656C8A
:100320002028303D3D64697361626C652900536526
:10033000742050504D206D696E696D756D20737914
:100340006E630053657420626561636F6E20696E31
:1003500074657276616C0053657420626561636FC9
:100360006E2064656C617900536574206265616319
:100370006F6E206672657175656E637920696E2097
:10038000487A3A20303D64697361626C652C205074
:10039000783D504D52206368616E6E656C20782CFC
:1003A0002046783D465253206368616E6E656C202E
:1003B00078005365742050574D2073746F7020641B
:1003C000656C61792028302064697361626C6564B2
:1003D0002C20312D323535203D3D20302E317320FB
:1003E0002D2035306D696E29005365742050504DB5
:1003F0002073746F702064656C61792028302064EC
:10040000697361626C65642C20312D323535203D75
:100410003D20302E3173202D2035306D696E29003E
:10042000536574206661696C736166652064656CF0
:1004300061792028302064697361626C65642C20C6
:10044000312D323535203D3D20302E3173202D2089
:1004500035306D696E29002A2A2A2A2A2A2A2A2A50
:100460002A2A2A2A2A2A2A2A2A2A2A2A2A2A2A2AEC
:100470002A2A2A2A0052582041636B6564202D20C5
:1004800072657665727420737563636573736675E0
:100490006C21002A2A2A2A2A2A2A2A2A2A2A2A2AAD
:1004A0002A2A2A2A2A2A2A2A2A2A2A2A2A2A2A2AAC
:1004B000002A2A2A2A2A2A2A2A2A2A2A2A2A2A2AC6
:1004C0002A2A2A2A2A2A2A2A2A2A2A2A2A2A00528E
:1004D000582041636B6564202D20757064617465DC
:1004E000207375636365737366756C21002A2A2A0D
:1004F0002A2A2A2A2A2A2A2A2A2A2A2A2A2A2A2A5C
:100500002A2A2A2A2A2A2A2A2A2A0056616C696457
:100510002063686F69636573206172653A205B319F
:100520005D2D5B31365D20286368616E6E656C20E1
:10053000312D31362900536574206F7574707574D0
:1005400020666F7220706F727420005B585D2061AE
:10055000626F7274206368616E67657320616E6498
:10056000206578697420525820636F6E6669670051
:100570005B535D20736176652073657474696E6783
:100580007320746F205258005B525D20726576654F
:1005900072742052582073657474696E6773207486
:1005A0006F2064656661756C747300557365206EA9
:1005B000756D62657273205B312D445D20746F2010
:1005C0006564697420706F727473205B452D515D92
:1005D00020666F722073657474696E677300202DD6
:1005E00020726563656976657220636F6E66696700
:1005F000757261746F722C20727820737720000AF4
:100600000A6F70656E4C52536E67200053657420FC
:1006100073657269616C2062617564726174653AB8
:10062000200056616C69642063686F696365733A82
:100630002031202D20342B34202F2032202D203823
:10064000202F2033202D20382B34202F2034202D14
:10065000203132202F2035202D2031322B34202FF5
:100660002036202D20313600536574204368616E9A
:100670006E656C20636F6E6669673A20005365741F
:100680002044617461726174652028302D32293AEA
:10069000200053657420486F70206368616E6E653A
:1006A0006C7320286D61782032342C207365706162
:1006B000726174656420627920636F6D6D61732966
:1006C0002076616C69642076616C75657320312DCC
:1006D0003235353A2000536574206368616E6E656B
:1006E0006C2073706163696E6720287831306B48C5
:1006F0007A293A200053657420524620706F77653E
:10070000722028302D37293A200053657420524634
:10071000206D6167696320286865782920652E67E8
:100720002E20307844454144463030443A2000532E
:1007300065742062617365206672657175656E63AC
:10074000792028696E20487A293A20005B5A5D207A
:10075000656E746572207265636569766572206383
:100760006F6E66696775726174696F6E2075746902
:100770006C79005B465D20646973706C61792061FF
:10078000637475616C206672657175656E63696509
:10079000732075736564005B525D2063616C6375E3
:1007A0006C6174652072616E646F6D206B65792079
:1007B000616E6420686F70206C697374005B495DC2
:1007C000207265696E697469616C697A6520736508
:1007D0007474696E677320746F20736B65746368DB
:1007E0002064656661756C7473005B585D2072658A
:1007F00076657274206368616E67657320616E64EC
:100800002065786974206D656E75005B535D20739B
:100810006176652073657474696E677320746F20E8
:10082000454550524F4D20616E64206578697420B3
:100830006D656E7500557365206E756D62657273BA
:10084000205B302D395D20746F20656469742070E1
:100850006172616D657465727300202D2053797328
:1008600074656D20636F6E66696775726174696F18
:100870006E000A0A6F70656E4C52536E672000510D
:1008800029204F7574707574206265666F726520DB
:100890006C696E6B20283D465329203A2000502970
:1008A00020536C617665206D6F64652028657870D3
:1008B0006572696D656E74616C293A20004F29205C
:1008C00054696D65642042494E44206174207374FC
:1008D000617274757020203A20004E292050504DCE
:1008E000206F7574707574206C696D69746564200F
:1008F000202020203A200044495341424C454400E6
:100900004D292050504D205253534920746F20637D
:1009100068616E6E656C202020203A20004C2920F2
:1009200050504D206D696E696D756D2073796E63E1
:10093000202875732920203A200044495341424C15
:100940004544004B29204661696C736166652062ED
:100950006561636F6E20696E74762E2028312D32AA
:10096000353573293A20004A29204661696C736144
:10097000666520626561636F6E2064656C617920D5
:1009800028302D323535203D3E20313073202D204A
:100990003135306D696E293A200049292046616958
:1009A0006C7361666520626561636F6E206672714B
:1009B0002E203A200048292050574D2073746F7024
:1009C0002064656C6179202020202020203A2000BE
:1009D00047292050504D2073746F702064656C61FE
:1009E00079202020202020203A200046292046611E
:1009F000696C736166652064656C617920202020D4
:100A00002020203A200050574D206368616E6E65AB
:100A10006C200066756E6374696F6E3A2000292041
:100A2000706F72742000506F776572546F776572C3
:100A300000445446205548462033322D62697420C4
:100A400031306368004F70656E4C52536E67525878
:100A5000206D696E6920342F36636800466C7974A6
:100A6000726F6E2F4F72616E6765525820554846FF
:100A70002038636800525820747970653A20004429
:100A8000697361626C656400487A00203D3D200016
:100A900043616C63756C61746564207061636B6540
:100AA0007420696E74657276616C3A200042292068
:100AB0004D6963726F202868616C66292050504D23
:100AC000202020203A00412920496E766572746505
:100AD000642050504D20696E20202020203A0030A4
:100AE00029204D7574652062757A7A657220286DAB
:100AF0006F73746C79293A003929205365726961E2
:100B00006C2062617564726174653A00736D617224
:100B100074506F7274004672536B79005472616E38
:100B200073706172656E740044697361626C6564B0
:100B30000038292054656C656D657472793A2020FF
:100B40002020202020003729204368616E6E656CCC
:100B500020636F6E6669673A202000362920446161
:100B60007461726174652028302D32293A2020206A
:100B700000352920486F70206368616E6E656C7364
:100B80003A2020202020003429204368616E6E65C1
:100B90006C2073706163696E673A202000332920EE
:100BA000524620706F7765722028302D37293A2001
:100BB0002020003229205246206D616769633A2067
:100BC0002020202020202020003129204261736530
:100BD000206672657175656E63793A202020000089
:100BE00000000700020100000304060000000000EE
:100BF00000000001020408102040800102040810D7
:100C00002001020408102004040404040404040263
:100C10000202020202030303030303000000002395
:100C2000002600290000000000250028002B0000FD
:100C3000000000240027002A0000722E11241FBE8D
:100C4000CFEFD8E0DEBFCDBF13E0A0E0B1E0E2EF30
:100C5000F2E602C005900D92A83CB107D9F716E064
:100C6000A8ECB3E001C01D92A239B107E1F71CE086
:100C7000CCE3DCE004C02297FE010E947B2FCA3344
:100C8000D107C9F70E94AE2E0C9477310C94000066
:100C900080917705813019F482E080937705809107
:100CA0007705833019F484E0809377050895A8953B
:100CB0000895DC01ED91FC910190F081E02D099502
:100CC00008952091780530917905382748E0C901C9
:100CD000880F991F37FF06C09C0151E2252750E17C
:100CE000352701C09C01415091F73093790520933D
:100CF0007805089588E380937A0580E092ECA1E07E
:100D0000B0E080937B0590937C05A0937D05B09324
:100D10007E0587E08093870580E091EAACEBB3E342
:100D200080937F0590938005A0938105B093820501
:100D300085E0809388058DEE9EEFADEABEED809351
:100D4000830590938405A0938505B0938605E9E813
:100D5000F5E080E090E0863028F4DC01AE54BC4F32
:100D60002C9101C020E0219301968831910599F7DB
:100D700082E08093A1058AE08093A205089580E037
:100D80009EECADEEB4E38093BF059093C005A093B5
:100D9000C105B093C20580E090E0A0E0B0E580938B
:100DA000C3059093C405A093C505B093C605E7ECB1
:100DB000F5E080E081938F5F8031E1F70895A0E056
:100DC000B0E0E5EEF6E00C94442FD82F0E942329E2
:100DD0006115710581059105C9F30E94E72F1092F5
:100DE0008305109284051092850510928605C4E053
:100DF000812C912C54018A94C0908305D090840555
:100E0000E0908505F0908605FE2CED2CDC2CCC24A2
:100E10000E94E22FA50194010E94232F6C0D7D1DDD
:100E20008E1D9F1D609383057093840580938505B7
:100E300090938605C15001F7DD2309F450C009E8FD
:100E400015E0E801A12CB12C62E3C62ED12CE12CD7
:100E5000F12C8881882309F442C0B39419F40E94CC
:100E60007A063DC00E94E22FA70196010E94232F1F
:100E7000E1E0E60FA9E8B5E08A2F801B8A1520F48F
:100E80008D918E13F9CFE9CF2091880530E0A0E154
:100E9000B7E20E94BB2E9B01AC01AE2FB0E00E94D6
:100EA000CA2E40907F05509080056090810570901B
:100EB0008205640D751D861D971D4090BF055090DD
:100EC000C0056090C1057090C205461657066806B9
:100ED000790618F2E993A39488E1A812BACFCDB7A6
:100EE000DEB7E0E10C94602F8436910520F4BC015C
:100EF00080E090E017C09C018E3B910528F42A55B4
:100F00003109AAE0B0E00CC0823D910528F4245BD1
:100F10003109A4E6B0E004C02D5C3109A8E5B2E0D7
:100F20000E94BB2EA4E6B0E09B01AC010E94CA2E39
:100F3000089590E08C599F4F0E947407089561E0D6
:100F400083E10E94D02960E083E10E94092A82E0C7
:100F50008093B00085E08093B10061E083E00E945F
:100F6000D02960E083E00E94092A0895A4E0B0E05F
:100F7000ECEBF7E00C94522F009749F19C0140E014
:100F800050E068E478EE81E090E00E94232F61E079
:100F900083E129833A834B835C830E94092A298158
:100FA000822F3A81932F4B81A42F5C81B52F8F3FE5
:100FB0009105A105B10529F020F08FEF90E0A0E0A8
:100FC000B0E08093B3008091B000806107C060E022
:100FD00083E10E94092A8091B0008F7E8093B00047
:100FE0002496E2E00C946E2F60E08CE00E94D02901
:100FF00061E08BE00E94D02961E08DE00E94D02961
:1010000060E082E00E94D02961E084E00E94D02963
:10101000089542E050E068E476E080E00E945328C2
:101020000895E3E0F0E089E080935700E491E670F2
:1010300081E0E63009F080E00895CF93DF93C82F78
:101040000E941108882381F0DFB781E08093760544
:10105000F8940E94570688E180936000C093600076
:10106000C1110E945706DFBFDF91CF9108958F9283
:101070009F92AF92BF92CF92DF92EF92FF92CF9367
:10108000FC01C0A5EC2FE770F0E0E658FC4FA08112
:10109000B0E0C7FF03C024E130E002C02FE030E041
:1010A000FC0197A183E1989FF0011124E25CFE4FBF
:1010B00080809180A280B380A20FB31F20E43FE123
:1010C0004DE750E00E94D52EA50194010E94012F0A
:1010D0008C2F887149F469017A01E0EDCE0EE7E0CA
:1010E000DE1EE11CF11C1BC0C7FF05C060E47AE8EE
:1010F0008CE29EE004C060E07EEE8AEB9BE069013A
:101100007A01F8EBCF0EFBE0DF1EE11CF11CA5011C
:1011100094010E94012FC20ED31EE41EF51EC701CA
:10112000B60169517C4F8F4F9F4F28EE33E040E06E
:1011300050E00E94012FA8EEB3E00E94CA2ECF918A
:10114000FF90EF90DF90CF90BF90AF909F908F90E7
:1011500008958F3F910551F048F0811522E09207E4
:1011600038F08115934030F482E0089580E00895CE
:1011700081E0089583E00895A0E0B0E0E2ECF8E0BB
:101180000C944D2FEB018A01B82FB695A0E0288171
:101190003981F80120832A813B8121832C813D8183
:1011A00022832E813F812383688179814A815B81FB
:1011B0002C813D81EE81FF819F2F9295990F990F90
:1011C000907C272F2370922B252F2370220F220F24
:1011D000922B232F23702295207F922BF80194834A
:1011E0000B5F1F4F2896AF5FBA1788F680FF24C0A9
:1011F000888199810E94A908D82E8A819B810E94AA
:10120000A908E82E8C819D810E94A908F82E8E8164
:101210009F810E94A908F0E4DF9EA001112490E1C3
:10122000E99E90011124242B282BE4E0FE9EB001BE
:101230001124262BF8012083CDB7DEB7E7E00C940C
:10124000692F803223E0920708F1883E23E092075D
:1012500040F48F519340E4E096958795EA95E1F745
:101260000895803D27E0920718F48C5D934008951F
:10127000883928E0920768F4885C974074E0969576
:1012800087957A95E1F78D509C4F089580E090E026
:1012900008958FEF93E008958C30910540F4A4E019
:1012A000880F991FAA95E1F7885D9C4F0895843FA8
:1012B00023E0920718F484529C4F0895811524E08E
:1012C000920740F48657934FF4E0880F991FFA95E0
:1012D000E1F7089580E998E008959C0136952795F7
:1012E00025753575821B930B9C012373337396957B
:1012F00087959695879583739373820F931F9C01AF
:1013000054E0369527955A95E1F7280F391F2F702D
:101310003F7041E051E0249FC001259F900D349F14
:10132000900D1124892F08952D98882319F000001D
:101330002B9A02C000002B9800002D9A00000895FF
:101340002D9A000083B12D98000082958170089538
:10135000CF93DF93D82F5C9A2D985C98C8E08D2F9F
:1013600080780E949409DD0FC150C9F72D98DF9154
:10137000CF9108958F770E94A8090895CF93DF93A6
:10138000D82FC8E08D2F80780E949409DD0FC150BE
:10139000C9F72D98DF91CF910895CF93DF932D98C2
:1013A000C8E080E0D82FDD0F0E94A0098D0FC1504A
:1013B000C9F7DF91CF9108950E94BA090E94CD0923
:1013C0005C9A0895A1E0B0E0E8EEF9E00C94522FA9
:1013D000806869830E94A8096981862F0E94BE09DE
:1013E0005C9A2196E2E00C946E2FCF93C091830516
:1013F000C827E82FF0E0E658FA4F678589E70E9492
:10140000E2096C2F8DE30E94E2096C2F82E40E94B6
:10141000E209CF91089586E20E94DC090895CF93F6
:10142000DF93EC016C818CE10E94E2096D818DE11A
:101430000E94E2096E818EE10E94E2096F8180E2E2
:101440000E94E209688581E20E94E209698582E2E0
:101450000E94E2096A8583E20E94E2096B8584E2C8
:101460000E94E2096C8585E20E94E2096D858AE2AC
:101470000E94E2096E858EE60E94E2096F858FE682
:101480000E94E209688980E70E94E209698981E790
:101490000E94E2096A8982E70E94E209DF91CF9106
:1014A0000895CF92DF92EF92FF92CF93DF936B017B
:1014B0007C01C11488E3D8068CE9E8068CE1F806C3
:1014C00028F5C701B60120E836E948E950E00E9456
:1014D000012FE901689760E879E687E69FEF0E94AF
:1014E000DD2E6C0D7D1D8E1D9F1DF2E0660F771F9A
:1014F000881F991FFA95D1F721E732E040E050E0CC
:101500000E94012FF22EE32E80E421C0C701B60114
:1015100020E03DE241E351E00E94012FE90168979C
:1015200060E073ED8EEC9EEF0E94DD2E6C0D7D1D54
:101530008E1D9F1D660F771F881F991F21E732E0C0
:1015400040E050E00E94012FF22EE32E80E66C2F47
:101550006F71680F85E70E94E2096E2D86E70E9491
:10156000E2096F2D87E70E94E209DF91CF91FF909A
:10157000EF90DF90CF900895682F8DE60E94E209EA
:1015800008958F929F92AF92BF92CF92DF92EF9287
:10159000FF92CF93DF93D82F83E00E94DC098093E2
:1015A000750584E00E94DC098093740560E086E0A4
:1015B0000E94E20961E087E00E94E2096FE789E0AA
:1015C0000E94E20965E08AE00E94E20962E18BE0A4
:1015D0000E94E20965E18CE00E94E2096DEF8DE076
:1015E0000E94E20960E08EE00E94E209DD2319F02A
:1015F0008BE291E008C02091A10533E1239FC00157
:101600001124825C9E4F0E940F0A6CE880E30E94C6
:10161000E2096FE082E30E94E20962E483E30E9450
:10162000E2098091A20587FF02C064E101C06AE07F
:1016300084E30E94E2096AE285E30E94E2096DE226
:1016400086E30E94E20964ED87E30E94E20960E01C
:1016500088E30E94E20960E089E30E94E209D11177
:1016600009C0C0908305D0908405E0908505F09076
:10167000860507C0C5E9CC2EC1ECDC2EED2CCEEDE5
:10168000FC2ECAE38F2C9924AA24BB24682D8C2F0E
:101690000E94E209682D85E08C0F0E94E209FE2C71
:1016A000ED2CDC2CCC24CF5FCE3361F76FEF83E4DD
:1016B0000E94E2096FEF84E40E94E2096FEF85E483
:1016C0000E94E2096FEF86E40E94E209DD2311F037
:1016D00066E002C0609187058DE60E94E20960E045
:1016E00089E70E94E209609188058AE70E94E20981
:1016F00060E083E70E94E20960E084E70E94E2097B
:10170000D11109C060917F0570918005809181059C
:101710009091820504C060E071EA8CEB93E30E9433
:10172000510ADF91CF91FF90EF90DF90CF90BF9063
:10173000AF909F908F90089561E087E00E94E2094A
:1017400064E28EE70E94E20963E088E00E94E20919
:1017500060E088E00E94E20965E087E00E94E2091B
:1017600062E085E00E94E20983E00E94DC09809348
:10177000750584E00E94DC0980937405089583E078
:101780000E94DC098093750584E00E94DC09809347
:10179000740561E087E00E94E2096AE070E080E0A1
:1017A00090E00E9446290E949C0B00000895CF9271
:1017B000DF92FF920F931F93CF93DF931F92CDB7CA
:1017C000DEB7082F162F8EE399830E94E209F02ED0
:1017D000C02E9981D92E8C2D8F19811738F4F601DE
:1017E00061916F018FE70E94E209F5CF64E085E027
:1017F0000E94E20983E00E94DC098093750584E081
:101800000E94DC09809374050E942329609370056F
:1018100070937105809372059093730569E087E07A
:101820000E94E20981E0809377050F90DF91CF91CC
:101830001F910F91FF90DF90CF9008950F931F930A
:101840000E94D70B80917705813099F40E9423295B
:10185000009170051091710520917205309173050A
:10186000601B710B820B930B603A764881409105A7
:1018700048F380917705813031F46EE971E086EEAE
:1018800095E00E940F2B1F910F9108950F931F93C6
:1018900080917705823021F41092770581E020C095
:1018A000809177058130D9F40E9423290091700539
:1018B000109171052091720530917305601B710BB9
:1018C000820B930B613A76488140910540F061E0CC
:1018D00087E00E94E2091092770582E001C080E073
:1018E0001F910F910895CF93DF93EC014AE050E0F0
:1018F0006D2F70E086EE95E00E94DD2B6EE286EEA5
:1019000095E00E94E12ABE0184E0769567958A956C
:10191000E1F76F7077274AE050E086EE95E00E948D
:10192000DD2B6EE286EE95E00E94E12ABE016F702B
:1019300077274AE050E086EE95E00E94DD2BDF91AC
:10194000CF910895D82FC0E0CD1790F45E9A409AB9
:1019500064E670E080E090E00E9446295E9840983E
:1019600064E670E080E090E00E944629CF5FECCF13
:101970006CE271E080E090E00E944629E4CF0F9392
:101980001F93CF93DF93EC01062F15E0115051F018
:10199000CE010E945E31081741F0602FCE010E94F7
:1019A0006631F4CF82E00E94A20CDF91CF911F91AB
:1019B0000F910895A0E0B0E0E0EEFCE00C94442F1D
:1019C000482E562EC0E0D0E0612C712CE12CF12C79
:1019D00000E010E041100CC06090D80586E4689EDD
:1019E0003001112459E1E52EF12C0EEB15E01EC05B
:1019F00091E049120FC06090D805E6E46E9E300178
:101A00001124FBE16F0E711C49E2E42EF12C0AE770
:101A100015E00CC082E0481209C028E1622E77244C
:101A20007394EE24E394F12C07ED15E043018C0E42
:101A30009D1E10927905109278053401A62CA818E5
:101A4000B12CC30101966C01AE14BF04A8F4A00E22
:101A5000B11E511006C0C3010E945E31F5018083A2
:101A600005C0F5016081C3010E94BF0CF5018081B2
:101A70000E9461063601E2CFC301511018C0C301B4
:101A80000E945E31B82EC6010E945E312B2D30E0DF
:101A9000322F2227282B8091780590917905821783
:101AA000930779F4C0E0D0E05524539493CF3601E6
:101AB000609179050E94BF0C60917805C6010E9473
:101AC000BF0CC05EDE4FC13E92E0D90708F482CF62
:101AD000852DCDB7DEB7E0E10C94602F61E082E0A8
:101AE0000E94DA0C089560E082E00E94DA0C809196
:101AF000D705853020F01092D7050E946E0D809199
:101B0000D7058093D805089561E080E00E94DA0C43
:101B100061E081E00E94DA0C089560E080E00E94BC
:101B2000DA0C882351F060E081E00E94DA0C88230F
:101B300021F080917A05883349F00E94BF060E9407
:101B40007A0681E00E94DF060E94840D08958823B2
:101B500019F06AEA71E002C06EEA71E086EE95E083
:101B60000E940F2B0895FF920F931F93CF93DF9343
:101B700069EC7BE086EE95E00E94BB2A40917F05F0
:101B80005091800560918105709182052AE030E0D6
:101B900086EE95E00E94E42B63EB7BE086EE95E019
:101BA0000E94BB2A40918305509184056091850570
:101BB0007091860520E130E086EE95E00E94E42BEE
:101BC0006DE97BE086EE95E00E94BB2A4AE050E09A
:101BD0006091870586EE95E00E940C2C67E87BE01B
:101BE00086EE95E00E94BB2A4AE050E060918805AD
:101BF00086EE95E00E940C2C61E77BE086EE95E096
:101C00000E94BB2AC9E8D5E0F12C8E018881882387
:101C1000A9F0FF2031F061EB71E086EE95E00E94C3
:101C2000DE2A21964AE050E0F801608186EE95E0D8
:101C30000E94D52BF394F8E1FF12E7CF86EE95E0F2
:101C40000E94E92A6BE57BE086EE95E00E94BB2AC4
:101C50004AE050E06091A10586EE95E00E940C2CD0
:101C600066E47BE086EE95E00E94BB2AE091A20547
:101C7000E770F0E0EE0FFF1FEE57FC4F60817181BF
:101C800086EE95E00E940F2B61E37BE086EE95E007
:101C90000E94BB2A8091A2058871883069F028F4DF
:101CA000811113C068E27BE00CC0803141F08831C3
:101CB00061F46CE07BE005C06CE17BE002C066E1B2
:101CC0007BE086EE95E00E94FD2A68EF7AE086EEE2
:101CD00095E00E94BB2A40917B0550917C05609164
:101CE0007D0570917E052AE030E086EE95E00E9449
:101CF000E42B6FED7AE086EE95E00E94BB2A80919E
:101D0000C30580710E94A70D66EC7AE086EE95E02F
:101D10000E94BB2A8091C30580740E94A70D6DEAC2
:101D20007AE086EE95E00E94BB2A8091C30580721E
:101D30000E94A70D60E97AE086EE95E00E94BB2A3A
:101D40008AE795E00E943708AB01BC012AE030E049
:101D500086EE95E00E94C62B6BE87AE086EE95E071
:101D60000E94BB2A8AE795E00E9437089B01AC01DC
:101D700060E472E48FE090E00E94012FBA01A901B3
:101D80002AE030E086EE95E00E94C62B68E87AE013
:101D900086EE95E00E94FD2ACDB7DEB7E5E00C9413
:101DA0006B2F8F929F92AF92BF92CF92DF92EF9262
:101DB000FF92811107C06FE77AE086EE95E00E94FE
:101DC000FD2A2FC090E00E94740724E630E040E036
:101DD00050E00E94012FCA01B9012AE030E040E042
:101DE00050E00E94012F49015A016B017C012AE059
:101DF00030E0B501A40186EE95E00E94C62B6EE2AC
:101E000086EE95E00E94E12A2AE030E0B701A601C3
:101E100086EE95E00E94C62B63E786EE95E00E9471
:101E2000212BFF90EF90DF90CF90BF90AF909F90CD
:101E30008F9008951F93CF93DF9365E77AE086EE46
:101E400095E00E94BB2A8091A305813041F46CE5A6
:101E50007AE086EE95E00E94FD2A10E050C08230C4
:101E600019F465E47AE0F5CF843019F461E37AE09F
:101E7000F0CF853091F766E27AE0EBCFC12FD0E06A
:101E8000C930D1050CF441C068E3610F86EE95E0DE
:101E90000E94E12A6EE17AE086EE95E00E94BB2A7C
:101EA000BE016F5F7F4F4AE050E086EE95E00E94F2
:101EB000A52B63E17AE086EE95E00E94BB2ACD5522
:101EC000DA4FE981E03218F566E07AE086EE95E0D7
:101ED0000E94BB2A8981803130F06DE673E086EE86
:101EE00095E00E94DE2A69816F7070E06F5F7F4F1E
:101EF0004AE050E086EE95E00E94AE2B1F5F809195
:101F00004C05181708F4BACF0FC061E3BECFEF70CD
:101F1000F0E0EE0FFF1FEE56FC4F6081718186EE00
:101F200095E00E940F2BEACF6BEE79E086EE95E00C
:101F30000E94BB2A8091BB050E94D10E60ED79E022
:101F400086EE95E00E94BB2A8091BC050E94D10ECE
:101F500065EB79E086EE95E00E94BB2A8091BD0595
:101F60000E94D10E6AE979E086EE95E00E94BB2AD4
:101F70004091B3055091B4056091B5057091B605D7
:101F8000411551056105710539F12AE030E086EE11
:101F900095E00E94E42B67E679E086EE95E00E94EA
:101FA000BB2A8091B7050E949907AB01BC012AE0CA
:101FB00030E086EE95E00E94E42B63E479E086EE63
:101FC00095E00E94BB2A4AE050E06091B80586EE99
:101FD00095E00E940C2C06C06AE379E086EE95E05D
:101FE0000E94FD2A6DE179E086EE95E00E94BB2A11
:101FF0006091B9057091BA054AE050E086EE95E02F
:102000000E94F62B60E079E086EE95E00E94BB2A04
:102010006091B205603450F470E06F5F7F4F4AE02A
:1020200050E086EE95E00E94AE2B06C067EF78E0A8
:1020300086EE95E00E94FD2A6AED78E086EE95E056
:102040000E94BB2A8091B10580FF03C063EB71E061
:1020500002C067EB71E086EE95E00E940F2B6DEBFE
:1020600078E086EE95E00E94BB2A8091B1058270EF
:102070000E94A70D6EE978E086EE95E00E94BB2AEB
:102080008091B10584700E94A70D6FE778E086EE1D
:1020900095E00E94BB2A8091B10588700E94A70D2F
:1020A000DF91CF911F9108950F931F93CF93DF93EB
:1020B000209149052F3FA9F56FEF75E086EE95E079
:1020C0000E94BB2A88E893E00E94730C6EED75E0D5
:1020D00086EE95E00E94BB2A80914A0590914B05BF
:1020E0000E94730C6BEA75E086EE95E00E94FD2A73
:1020F00068E875E086EE95E00E94FD2A60E775E0ED
:1021000086EE95E00E94FD2A6BE475E086EE95E090
:102110000E94FD2A86EE95E00E94E92A0E941A0F8D
:1021200068C012160CF065C0332727FD30958091EA
:102130004C0590E0821793070CF45BC066E375E0F2
:1021400086EE95E00E94BB2A60914905772767FDDE
:1021500070954AE050E086EE95E00E94AE2B6BE071
:1021600075E086EE95E00E94BB2A10E008E28091BF
:102170004D051817D0F5C12FD0E0CC0FDD1FC25B85
:10218000DA4F288130E080914905992787FD9095A5
:1021900001972817390739F56BEB71E086EE95E06A
:1021A0000E94DE2A4AE050E0602F86EE95E00E9411
:1021B000D52B6FEB71E086EE95E00E94DE2AE98177
:1021C000EF70F0E0EE0FFF1FEE56FC4F6081718163
:1021D00086EE95E00E94DE2A63EC71E086EE95E0E3
:1021E0000E94DE2A0F5F1F5FC2CF86EE95E00E943D
:1021F000E92ADF91CF911F910F910895FF920F93DC
:102200001F93CF93DF93C9E8D5E0F12C8E0188812D
:102210008823D1F165EC71E086EE95E00E94DE2A1C
:102220004AE050E06F2D86EE95E00E94D52B62EDDE
:1022300071E086EE95E00E94DE2A2196F801208169
:1022400030E0A0E1B7E20E94BB2E9B01AC01A0915F
:102250008805B0E00E94CA2EAB01BC0180917F05C9
:1022600090918005A0918105B0918205480F591F7A
:102270006A1F7B1F2AE030E086EE95E00E94E42B87
:10228000F394F8E1FF12C2CFCDB7DEB7E5E00C94CE
:102290006B2F1092E30485E6E4EEF4E0DF011D927B
:1022A0008A95E9F70895CF93C82F8F3719F08830B2
:1022B00009F045C0E091E304EE23D9F1E150E09349
:1022C000E304F0E0EC51FB4F10826DE070E086EE2D
:1022D00095E00E945906C0E08091E304C81760F4BD
:1022E000EC2FF0E0EC51FB4F608170E086EE95E062
:1022F0000E945906CF5FF0CF60E270E086EE95E075
:102300000E9459066DE070E086EE95E00E94590645
:10231000C0E08091E304C81778F5EC2FF0E0EC51B1
:10232000FB4F608170E086EE95E00E945906CF5F1A
:10233000F0CF67E086EE95E00E94E12A1DC08B3168
:1023400019F40E9449111AC08D30C1F08A30B1F0E1
:102350008091E304843668F76C2F70E086EE95E098
:102360000E945906E091E30481E08E0F8093E3041C
:10237000F0E0EC51FB4FC08380E001C081E0CF91E1
:102380000895CF93C82F0E9423296093CC047093A3
:10239000CD048093CE049093CF04C093E104CC236A
:1023A00029F040E051EE60E070E004C040E855E202
:1023B00060E070E086EE95E00E946B2DCF9108956D
:1023C0009091D004492F4F7050E0BA016F5F7F4F5A
:1023D000292F30E0E4E035952795EA95E1F762177B
:1023E000730759F0FA01EF52FB4F808381E0890FA8
:1023F0008F70907F892B8093D00408956EE770E0F2
:1024000086EE95E00E9459060895A3E1B1E0EBE065
:10241000F2E10C94452FE9E8F5E0712C81918823D5
:1024200021F0739428E17212F9CF66ED71E086EE27
:1024300095E00E940F2B4AE050E0672D86EE95E074
:102440000E940C2C80E00E94C10A0E949C0B8E010D
:102450000E5F1F4FC12CD12C7601C39466246A9461
:102460005C2C0E9417294B015C012091880530E00B
:10247000A0E1B7E20E94BB2E9B01AC01C701B601EF
:102480000E94DD2E20917F053091800540918105CD
:1024900050918205620F731F841F951F2091BF0505
:1024A0003091C0054091C1055091C20526173707EC
:1024B0004807590718F4F801608229C08C2D0E9442
:1024C000F50961E070E080E090E00E944629F801A3
:1024D00010820E941729681979098A099B09643FAB
:1024E00071408105910540F40E940B0AF80190812A
:1024F000981778F78083EDCF50FE05C05D9841981E
:102500005E9A409A04C05D9A419A5E9840982FEF77
:10251000C21AD20AE20AF20A0F5F1F4F8FEFC816E3
:10252000D104E104F10409F09BCFCE019395FC01A5
:10253000D82E7FEF68EC2E2F281B271510F051E0C6
:1025400056C0DE01129651E02FEF41E03D91321767
:1025500010F0322F01C0452F5F5F5F3F11F0232F36
:10256000F5CF4193242F30E0A1E0B0E0AC0FBD1FC8
:10257000A20FB31F5C93413079F0DE01A20FB31FAD
:102580005C93423049F0AFEFBFEFAC0FBD1FA20F1D
:10259000B31F6C934E3F78F6A2E0B0E0AC0FBD1FC6
:1025A000A20FB31F7C934D3F30F6A3E0B0E0AC0F19
:1025B000BD1FA20FB31F6C93BECF452F242F30E059
:1025C000FC01E20FF31F6081AFEFB0E0AC0FBD1F65
:1025D000A20FB31F2C91621748F44150DC01A40FE5
:1025E000B11D2C9120836C934111E8CF5F5F57158B
:1025F00020F3372D369520E0231770F4DC01A20F6D
:10260000B11D4C91522F530FFC01E50FF11D50816C
:102610005C9340832E5FF0CFF9E8EF2EF5E0FF2EBC
:102620008C01802F8D19871598F4F801C1908F01C6
:102630004AE050E06C2D86EE95E00E94D52B6CE2CE
:1026400086EE95E00E94E12AF701C1927F01E9CF71
:1026500086EE95E00E94E92A81E0CD5EDE4FEFE054
:102660000C94612F1F920F920FB60F9211241F939B
:102670002F933F934F935F936F937F938F939F938A
:10268000AF93BF93CF93DF93EF93FF93C0918600F7
:10269000D091870080918704909188042091A904AB
:1026A000211155C09E01281B390B8091C3059091C3
:1026B000C405A091C505B091C60585FD02C036953B
:1026C0002795253C49E03407B8F140910A0150E0D4
:1026D00060E070E02CE1B695A795979587952A95CF
:1026E000D1F70097A105B10521F481E090E0A0E0C9
:1026F000B0E084179507A607B707D8F480910A01C0
:102700008F3FB9F040E080910A01481780F4842F90
:1027100090E0880F991FFC01E757FB4F2081318122
:10272000FC01E55FFE4F318320834F5FECCF1092B9
:10273000AA0410920A010BC02D3B82E0380720F05A
:1027400080910A018031D8F08FEF80930A01D093F5
:102750008804C0938704FF91EF91DF91CF91BF91DF
:10276000AF919F918F917F916F915F914F913F9129
:102770002F911F910F900FBE0F901F9018951091E1
:102780000A0181E0810F80930A01C9010E94210999
:10279000E12FF0E0EE0FFF1FE757FB4F918380839F
:1027A000D6CF83E0809380008AE980938100809176
:1027B000C30586FD05C080918100806480938100FF
:1027C0008FEF9FEF909389008093880080916F0036
:1027D000806280936F0008950E94730D8091D805E8
:1027E000843011F41092D80508956F3018F0869552
:1027F0008058089589E0689F802D11240895A0E0F5
:10280000B0E0E5E0F4E10C944C2FC82F0E9423299E
:10281000009138041091390420913A0430913B041E
:102820006B017C01C01AD10AE20AF30A9701860102
:1028300049E8C41643E1D406E104F10410F0109213
:102840003C04609338047093390480933A04909365
:102850003B042091A9048FEF820F8230E8F5E091CC
:102860003C04EE2309F46EC1E13011F482E0D8C1DA
:10287000E03178F581E08E0F80933C04F0E0E7577B
:10288000FB4FC083803109F0D4C1EBE8F4E0213084
:1028900029F4A181A695A695808108C080819181A7
:1028A000A92FA695A695A69596958795A03148F44B
:1028B000B0E090E0AA0FBB1FA55FBE4F11969C939E
:1028C0008E931092AA04329684E0E939F807F9F65B
:1028D000B0C110923C04ADC1233009F023C1E09196
:1028E0003C04E11118C0CF3009F011C10E94172932
:1028F0000091B7041091B8042091B9043091BA0442
:10290000601B710B820B930B623071058105910581
:1029100008F089C1FCC0E83148F481E08E0F809353
:102920003C04F0E0E857FB4FC083F1C0E83109F008
:10293000ECC0C111EAC040E050E0ABE0CA01B3E036
:10294000880F991FBA95E1F7A49F9001A59F300DBC
:102950001124F901E757FB4F6081E1817E2F7770E9
:1029600075956795FC01EE0FFF1FE55FFE4F7183C4
:102970006083F901E657FB4FB081B695B695B695E1
:10298000E181FE2FF295FF0FF07E6F2F6B2BE69506
:10299000E695E6957E2F777075956795FC01EE0FAD
:1029A000FF1FE35FFE4F71836083F901E557FB4F23
:1029B000B081B295B695B695B370C181DC2FDD0FAD
:1029C000DD0F6D2F6B2BC295C695C695C370E28146
:1029D000E170EE0FEE0F7E2F7C2B75956795FC0155
:1029E000EE0FFF1FE15FFE4F71836083F901E35734
:1029F000FB4FB081B695E181FE2FF795FF27F79544
:102A00006F2F6B2BE6957E2F777075956795FC0180
:102A1000EE0FFF1FEF5EFE4F71836083F901E257F7
:102A2000FB4FB081B295BF70E181FE2FF295F07F30
:102A30006F2F6B2BE295EF707E2F777075956795F2
:102A4000FC01EE0FFF1FED5EFE4F71836083F90105
:102A5000E157FB4FB081BB1FBB27BB1FC181DC2FE0
:102A6000DD0F6D2F6B2BCC1FCC27CC1FE281E370C9
:102A7000EE0F7E2F7C2B75956795FC01EE0FFF1FE7
:102A8000EB5EFE4F71836083F901EF56FB4FB0811F
:102A9000B695B695E181FE2FF295FF0FFF0FF07C02
:102AA0006F2F6B2BE695E6957E2F77707595679562
:102AB000FC01EE0FFF1FE95EFE4F71836083F90199
:102AC000EE56FB4F20812295269527703181E32F0A
:102AD000EE0FEE0FEE0F6E2F622B732F7295769521
:102AE000777075956795FC01EE0FFF1FE75EFE4F4F
:102AF000718360834F5F5F4F4230510509F01ECFF5
:102B000080919F0483FF1092AA0410923C040E94BB
:102B100017296093B7047093B8048093B904909315
:102B2000BA0487C0243009F084C060913C0461116C
:102B30000BC0C83AB1F4109279051092780588EA72
:102B40000E94610681E06CC0613019F4C0933704C3
:102B500004C0623031F4C09336048C2F0E946106A9
:102B60005AC0E09136042E2F30E0220F331F462F3B
:102B700050E0C9010296841795073CF0633268F76C
:102B8000FA01EA57FB4FC083E8CF2D5F3F4F8C2FF0
:102B900090E060917805709179054217530749F4E8
:102BA000982F882786279727909379058093780513
:102BB00032C06817790769F580913704813049F58B
:102BC000E13118F080E180933604F0903604CAE8D1
:102BD000D4E000E010E00F15D0F4FE0131978081C1
:102BE00090E0982F88272881822B63E0969587951F
:102BF0006A95E1F70E942109F801EE0FFF1FE55FDA
:102C0000FE4F918380830F5F1F4F2296E4CF109277
:102C1000AA0410923C0480913C04882351F08F5FF9
:102C200080933C0406C080913C048F5F80933C04F9
:102C30006ECFCDB7DEB7E8E00C94682FE82FF0E058
:102C4000E254FA4FE185E03150F4F894F0E0EE0FF1
:102C5000FF1FE55FFE4F80819181789408958EE09B
:102C60008E0F8B3058F4F0E0E25FF10924E62E9FDE
:102C7000C0012F9F900D11240C960895E03FF1F0B4
:102C800028F4E03161F0E13161F006C0ED3F81F000
:102C9000EE3F89F0E13F49F080E092E0089582E163
:102CA00001C083E10E94652A089586E090E00895BE
:102CB0008AEF93E008958FEF93E0089580E090E02D
:102CC0000895A2E2B0E0E7E6F6E10C94422F9E01FF
:102CD0002F5F3F4F80E1D9011D928A95E9F764E0AB
:102CE00072E086EE95E029A33AA30E940F2B0E9482
:102CF000BF0B1D8A1E8A1F8A188E312C212C00E0E2
:102D0000812C912C5401412C74E7572E7BE8672EBF
:102D100072E3772EE0E5CE2EE3ECDE2EE12CF12CF3
:102D200084EF91E0A0E0B0E08D8F9E8FAF8FB8A3CD
:102D300080E09EECADEEB4E3898F9A8FAB8FBC8FB1
:102D400080E094E7ABE8B2E3898B9A8BAB8BBC8BCA
:102D500086EE95E00E94232C892B09F4E1C086EED3
:102D600095E00E94502C9C0133272C32310509F448
:102D700042C0ACF42332310509F0ABC019821A828B
:102D80001B821C821D821E821F82188619861A864B
:102D90001B861C861D861E861F86188A60C02434EA
:102DA000310529F02335310509F4B2C092C064E43D
:102DB00086EE95E00E94E12A2AE030E040E054E708
:102DC0006BE872E386EE95E00E946F2B6CE286EE74
:102DD00095E00E94E12A2AE030E040E05EEC6DEEF2
:102DE00074E386EE95E00E946F2B6CE286EE95E030
:102DF0000E94212BADCF0F5F043009F0A9CF2981AC
:102E00003A814B815C81A8EEB3E00E94CA2E698BA7
:102E10007A8B8B8B9C8B2D813E814F8158850E94B4
:102E2000CA2E698F7A8F8B8F9C8F29853A854B8527
:102E30005C852D8F3E8F4F8F58A32D853E854F8506
:102E400058890E94CA2E6B017C0160323EE47307F0
:102E50008105910530F462E38CE10E94E20900E013
:102E600077CF603345E774078105910510F462E27E
:102E7000F3CF60345CE975078105910510F466E2D3
:102E8000EBCF80E5C81683ECD806E104F10410F41A
:102E900062E1E2CF90E6C9169AEED906E104F104A8
:102EA00010F465E1D9CFA0E7CA16A1E1DA06A1E0E6
:102EB000EA06F10410F461E0CFCFB0EACB16B6E831
:102EC000DB06B1E0EB06F10410F463E0C5CF65E08A
:102ED000C3CF10ED180F1A3008F03ACFE1E0F0E060
:102EE000EC0FFD1F24E0029FE00DF11D1124208155
:102EF000318142815381AAE0B0E00E94CA2E610F65
:102F0000711D811D911D608371838283938320CF06
:102F100049885A886B887C88812C912C540118CF61
:102F200081149104A104B10489F4C301B2010E9487
:102F3000510A61E070E080E090E00E9446291D8A1D
:102F40001E8A1F8A188E312C22242A948D8D9E8DE4
:102F5000AF8DB8A188169906AA06BB06D0F40E94C8
:102F60000B0A2D893E894F89588D280F311D411D2F
:102F7000511D2D8B3E8B4F8B588F381608F4382EF1
:102F8000821508F4282E3FEF831A930AA30AB30A86
:102F900056C0C301B20128EE33E040E050E00E9489
:102FA000012FBA01A9012AE030E086EE95E00E94E7
:102FB000C62B6CE286EE95E00E94E12A4AE050E0E2
:102FC000632D86EE95E00E94D52B6CE286EE95E0AF
:102FD0000E94E12A6D897E898F89988DA5019401CF
:102FE0000E94012FBA01A9012AE030E086EE95E0A7
:102FF0000E94C62B6CE286EE95E00E94E12A4AE030
:1030000050E0622D86EE95E00E94D52B6CE286EEB4
:1030100095E00E94212B4C0C5D1C6E1C7F1C898D41
:103020009A8DAB8DBC8D84159505A605B70520F44A
:1030300049885A886B887C88812C912C5401298975
:103040003A894B895C89283E33404105510509F096
:103050007FCEA296E2E10C945E2FACE1B0E0E3E318
:10306000F8E10C944C2F0E9423296B017C0181E034
:103070000E94C10A14E703E0198361E0CE010196C2
:103080000E941E0C009377050E949C0B6AEF70E073
:1030900080E090E00E94462980917705833089F492
:1030A00086EE95E00E94232C892B59F40E94232957
:1030B0006C197D098E099F096038734C894C9140C9
:1030C000D8F280917705833009F44FC08FE70E94D2
:1030D000BA090E94CD098983843511F083E05CC070
:1030E0000E94CD0910924A0580934B050E94CD099C
:1030F00020914A0530914B05280F311D30934B0527
:1031000020934A050E94CD0980934C050E94CD0969
:1031100080934D05813110F7F12C0F2D10E0809137
:103120004D0590E0880F991F0817190740F40E9479
:10313000CD09F801E25BFA4F8083F394EECF80E78C
:10314000898361E0CE0101960E941E0C83E080938A
:1031500077050E949C0B62E370E080E090E00E94A3
:10316000462980917705833011F482E015C08FE7FE
:103170000E94BA090E94CD098983803509F0AECF3B
:1031800003EA15E00E94CD09F80181938F01F5E073
:103190000E3B1F07B9F781E06C96E8E00C94682FAE
:1031A00080914905992787FD9095A92FB92FFC019A
:1031B0003196EB30F10508F066C0EC5CFF4F0C94E3
:1031C000792F62E778E086EE95E00E94FD2A88E894
:1031D00093E00E94730C6AE578E086EE95E00E9429
:1031E000FD2A65E378E086EE95E00E94FD2A6BE01B
:1031F00078E086EE95E00E94FD2A6AEE77E086EEA2
:1032000095E00E94FD2A6DEB77E086EE95E00E9446
:10321000FD2A67E977E086EE95E00E94FD2A63E7E4
:1032200077E086EE95E00E94FD2A6CE477E086EE7A
:1032300095E00E94FD2A86EE95E00E94E92A0E9410
:10324000B30D21C06FE277E01AC06AE077E017C0E3
:1032500065EF76E014C066ED76E011C062E976E0D5
:103260000EC06DE776E00BC068E676E086EE95E08E
:103270000E94FD2A62E276E002C06CE076E086EE13
:1032800095E00E94FD2A6AE070E080E090E00E94F4
:10329000462986EE95E00E94232C892B29F086EEA4
:1032A00095E00E94502CF5CF0895ACE1B0E0EBE53D
:1032B000F9E10C944C2F909149059F3F09F023C1EF
:1032C000482F50E0FA013A97EF36F10508F00FC1A8
:1032D000E15CFF4F0C94792F61E172E0A0C06DE1D9
:1032E00072E086EE95E00E940F2B85E789838BE1E3
:1032F000E3EAF5E0DE01129601900D928A95E1F77E
:103300006CE1CE0101960E941E0C0E949C0B83E092
:103310008093770568EC70E080E090E00E94462999
:1033200080917705843009F0E2C08FE70E94BA09E6
:103330000E94CD098983853509F0D9C06DEE74E00E
:1033400086EE95E00E94FD2A6FEC74E086EE95E033
:103350000E94FD2A61EB74E096C065E372E086EEA0
:1033600095E00E940F2B89E6898361E0CE010196EA
:103370000E941E0C0E949C0B83E08093770568ECF2
:1033800070E080E090E00E944629809177058430CB
:1033900009F0ADC08FE70E94BA090E94CD09898368
:1033A0008E010E5F1F4F7E014DE1E40EF11C0E9465
:1033B000CD09F80181938F01EE15FF05C1F78BE16F
:1033C000FE013296A3EAB5E001900D928A95E1F7ED
:1033D0008981893409F08BC063E974E086EE95E059
:1033E0000E94FD2A65E774E086EE95E00E94FD2AC2
:1033F00067E574E048C06FE472E086EE95E00E94F5
:103400000F2B8EEF8093490572C0805287508053F6
:1034100090914C05981708F066C06EE572E086EE54
:1034200095E00E940F2B63C084E18093490560E220
:1034300074E029C085E18093490569EE73E023C0FB
:1034400086E18093490562EB73E01DC087E18093BC
:10345000490568E673E017C088E18093490567E590
:1034600073E011C089E18093490563E473E00BC008
:103470008AE1809349056EE273E005C08BE1809399
:10348000490566E073E086EE95E00E94FD2A2FC0B4
:103490006CEE72E086EE95E00E94FD2A8091B10507
:1034A00091E01DC066ED72E086EE95E00E94FD2A77
:1034B0008091B10592E013C061EC72E086EE95E078
:1034C0000E94FD2A8091B10594E009C066EA72E08D
:1034D00086EE95E00E94FD2A8091B10598E089274B
:1034E0008093B1058FEF809349050E94541086EEBA
:1034F00095E00E94232C892B09F45AC186EE95E0B1
:103500000E94502CF4CF0E945311882309F450C11B
:103510008091E304811104C08FEF8093490540C17D
:1035200040E050E060E070E084EE94E00E94F02F14
:1035300040914905042F112707FD1095212F312FA8
:10354000F8013197EB31F10508F01AC1E255FF4F50
:103550000C94792F552747FD509520914C0530E06C
:10356000241735070CF40CC18B019C010150110983
:1035700021093109003211052105310558F0C090AB
:103580004D05EFE4F5E0F12CD12CA8E2EA2E4150F4
:1035900051090FC0FA01ED55FA4F61506083D8C050
:1035A000DF0111972C9130E02417350729F0F394AF
:1035B0003296FC10F5CFCAC00E2D10E020E030E0AE
:1035C000061717072807390741F42081DA01AD559E
:1035D000BA4F11962C93DD24D394E394E8CF6F3F38
:1035E00071058105910511F008F0CAC06093BB0513
:1035F000AFC06F3F71058105910511F008F0C0C0A3
:103600006093BC05A5C06F3F71058105910511F060
:1036100008F0B6C06093BD059BC02091E404206211
:103620002037E9F440E050E060E070E085EE94E09F
:103630000E94F02F9B01AC01DC01CB010197A10995
:10364000B1090897A105B10508F0ADC0A4EDB0E33C
:103650000E94CA2E6A5E7C4A8A46954E24C026364F
:10366000E9F440E050E060E070E085EE94E00E9414
:10367000F02F9B01AC01DC01CB010197A109B1093D
:103680000797A105B10508F08EC0A8EAB1E60E942F
:10369000CA2E645E7C438E46944E05C0611571054A
:1036A0008105910571F08B019C0114572B48324321
:1036B0000130FAE51F07F2E62F07F2E03F0708F0B6
:1036C0005FC06093B3057093B4058093B505909384
:1036D000B6053EC06F3F71058105910511F008F0F8
:1036E0004FC06093B70534C08B019C010150110994
:1036F000210931090F3F11052105310508F040C0AE
:103700006093B80525C08B019C01045C1940210918
:1037100031090D344DE114072105310528F470936A
:10372000BA056093B90514C061157105810591054D
:1037300021F48FEF8093B2050BC0613471058105D0
:103740009105F0F461506093B20502C0DD20C1F034
:103750008091E20481111AC08091830590918405C3
:10376000A0918505B09186050196A11DB11D80939C
:10377000830590938405A0938505B093860506C0C4
:1037800060E772E086EE95E00E940F2B0E944911DF
:103790008FEF809349056AE086EE95E00E94212B29
:1037A0000E94541005C061E070E080E090E07BCFA3
:1037B0006C96E8E00C94682F6AE572E086EE95E07E
:1037C0000E94FD2A62E472E086EE95E00E94FD2AE6
:1037D00086EE95E00E94232C892B31F086EE95E051
:1037E0000E94502C0E9455190E942D18823029F0F9
:1037F000833051F46DE072E002C064E272E086EE64
:1038000095E00E94FD2A08958FEF8093490510925C
:10381000E2040E945410809149058E3F69F086EEC3
:1038200095E00E94232C892BB1F386EE95E00E944F
:10383000502C0E945519EFCF08950F931F931091AC
:1038400049051F3F09F0D2C0893409F457C000F57B
:10385000883309F469C058F4803309F477C008F05C
:1038600061C08B3109F440C08132B1F1B9C08134FB
:1038700009F487C030F4893309F466C0803461F1FB
:10388000AFC0823409F48EC0863409F448C0A8C0A1
:10389000823609F487C078F4883531F128F482350E
:1038A000C1F18335E1F09CC08A3509F494C08136BA
:1038B00009F467C095C0823761F128F4863679F142
:1038C0008936E1F08DC0883779F08A3709F483C0F2
:1038D000833709F085C003C061E172E015C00E9422
:1038E000840D6EE872E004C00E948D0D68EA72E0FB
:1038F00086EE95E00E940F2B8EEF70C00E947A0634
:103900000E94BF0667EC72E086EE95E00E940F2BE6
:1039100067C081E00E94DF0660EE72E0F5CF0E9492
:10392000FE105EC080535AC06AEF71E086EE95E0EB
:103930000E94FD2A9091A20588E0890F8871977EE8
:10394000892B8093A2051AC089E048C067EE71E018
:1039500086EE95E00E94FD2A8091C3059091C405F2
:10396000A091C505B091C60520E182278093C305CB
:103970009093C405A093C505B093C605109349055F
:103980002FC061ED71E086EE95E00E94FD2A8091E6
:10399000C3059091C405A091C505B091C60540E44A
:1039A000842710C060EC71E086EE95E00E94FD2A4D
:1039B0008091C3059091C405A091C505B091C6053D
:1039C00020E282278093C3059093C405A093C50588
:1039D000B093C60502C00E94DC1B8FEF809349059F
:1039E000809149058E3F09F0D4C0DDC00E9453117B
:1039F000882309F4D8C08091E304811104C08FEFBB
:103A000080934905C6C040E050E060E070E084EE7D
:103A100094E00E94F02F00914905112707FD1095B1
:103A2000212F312FF8013197E930F10508F0B4C0AA
:103A3000E753FF4F0C94792F8B019C0101501447E1
:103A40002B4832430F3F19452246324008F0A4C0AC
:103A500060937F0570938005809381059093820524
:103A600077C0609383057093840580938505909358
:103A7000860581E08093E2046BC0683071058105A2
:103A8000910508F089C06093870562C08B019C0195
:103A900001501109210931090A30110521053105AB
:103AA00008F07AC06093880553C061EB71E084EE42
:103AB00094E00E942A3110E0009799F00E940431AE
:103AC000009779F0183130F4E12FF0E0E658FA4F22
:103AD00087871F5F61EB71E080E090E00E942A31F0
:103AE000EBCF1831A8F5E12FF0E0E658FA4F178632
:103AF0001F5FF7CF653071058105910508F04CC057
:103B00006093A10525C08B019C0101501109210979
:103B100031090630110521053105F0F52091A20586
:103B2000287F262B2093A20513C08B019C010150F6
:103B30001109210931090115124C2140310560F5A7
:103B400060937B0570937C0580937D0590937E0543
:103B50008091E204811113C08091830590918405C6
:103B6000A0918505B09186050196A11DB11D809398
:103B7000830590938405A0938505B09386050E94E4
:103B800049118FEF809349056AE086EE95E00E9427
:103B9000212B0E94D01807C060E772E086EE95E006
:103BA0000E940F2BECCF1F910F9108958FEF809300
:103BB00049051092E2040E94D018809149058E3F79
:103BC00069F086EE95E00E94232C892BB1F386EEF6
:103BD00095E00E94502C0E941D1CEFCF6AE070E01F
:103BE00080E090E00E94462986EE95E00E94232C1A
:103BF000892B29F086EE95E00E94502CF5CF089590
:103C0000CF93C82F682F86EE95E00E947D2C90916F
:103C10006E059C2790936E05CF910895A1E0B0E0CA
:103C2000E4E1FEE10C94522F99830E94001E9981D9
:103C3000892F0E94001E2196E2E00C946E2F1F93A4
:103C4000CF93DF93182FEB0110926E0565EB70E0B8
:103C500086EE95E00E94590662E670E086EE95E0F9
:103C60000E945906812F0E94001ECE010E940E1E46
:103C7000DF91CF911F91089560916E0586EE95E0DA
:103C80000E947D2C0895A1E2B0E0E9E4FEE10C94ED
:103C90004E2F7B018A018C3009F453C108F040C0DB
:103CA000863009F4BCC018F5833009F491C070F473
:103CB000813009F472C0823009F04AC26BE170E0D1
:103CC00082E00E941F1E03EA15E078C0843009F4E8
:103CD00087C0853009F03CC260914D0570E0660FE9
:103CE000771F85E00E941F1E0EE415E086C0893014
:103CF00009F4A7C070F4873009F49BC0883009F03C
:103D000027C261E070E088E00E941F1E8091D80504
:103D100025C28A3009F4CAC08B3009F4F2C018C237
:103D20008A3609F475C1D8F4873609F43AC138F4F3
:103D3000853609F40EC1863609F41FC109C28836DA
:103D400009F437C1893609F003C261E070E089E601
:103D50000E941F1E0E947A060E94BF06F7C18D3680
:103D600009F4D4C138F48B3609F491C18C3609F4C6
:103D70009AC1EEC18E3609F4DEC1873C09F0E8C174
:103D800061E070E087EC0E941F1E81E00E94001E2F
:103D90000E943C1E10926F05E5C169E270E081E06F
:103DA0000E941F1E0AE715E0F80181918F010E9411
:103DB000001EF5E0033A1F07B9F7D2C1F80181915F
:103DC0008F010E94001EF5E00E3B1F07B9F7C8C126
:103DD00061E070E083E00E941F1E0E942D18BEC1AA
:103DE00061E070E084E00E941F1E81E00E94001EDE
:103DF0000E943C1E0E946116B5C180914D0590E065
:103E0000880F991F98012E5435402817390708F05C
:103E1000A7C1F80181918F010E94001EEECF62E0E0
:103E200070E086E00E941F1E88E893E00E940E1E4C
:103E300097C161E070E087E00E941F1E80914C05F1
:103E40008DC186E6898361E0CE0101960E941E0C39
:103E50000E949C0B83E08093770568EC70E080E023
:103E600090E00E944629809177058430D9F48FE74D
:103E70000E94BA090E94CD098983863469F460E200
:103E800070E089E00E941F1E10E20E94CD090E948E
:103E9000001E1150D1F764C161E070E089E00E941A
:103EA0001F1E54C161E070E089E055C169E170E016
:103EB0008AE00E941F1E81E08093BE052091760556
:103EC0008091C3059091C405A091C505B091C60528
:103ED000222311F0806801C08F778093C3059093EF
:103EE000C405A093C505B093C6050EEB15E0F80117
:103EF00081918F010E94001EF5E0073D1F07B9F771
:103F00002FC161E270E08BE00E941F1E8091AA0425
:103F10008F3F39F08091AA0491E0980F9093AA0402
:103F200002C08091AA040E94001E10E0812F0E940E
:103F30001E160E944C090E940E1E1F5F1031B1F721
:103F40000FC161E070E08CE00E941F1E8091D705D8
:103F500005C161E070E085E60E941F1E89E2E81657
:103F6000F10409F0FAC0D801EAE7F5E08D918193F8
:103F700085E0E33AF807D1F7E9C061E070E086E652
:103F80000E941F1EEBE1EE16F10409F0E6C0D80115
:103F9000E3EAF5E08D91819385E0EE3BF807D1F7F8
:103FA000D5C061E070E087E60E941F1E0E94840D6C
:103FB000CDC061E070E088E60E941F1E85E789831E
:103FC0008BE1E3EAF5E0DE01129601900D928A950D
:103FD000E1F76CE1CE0101960E941E0C0E949C0B41
:103FE00083E08093770560E273E080E090E00E94D8
:103FF000462980917705843009F0AFC08FE70E9491
:10400000BA090E94CD098983853509F0A6C09EC0F2
:1040100061E070E08AE60E941F1E89E6898361E004
:10402000CE0101960E941E0C0E949C0B83E080939F
:10403000770560E273E080E090E00E94462980917D
:104040007705843009F089C08FE70E94BA090E9481
:10405000CD0989838E010E5F1F4F7E01EDE1EE0ECB
:10406000F11C0E94CD09F80181938F01EE15FF0527
:10407000C1F78BE1FE013296A3EAB5E001900D9203
:104080008A95E1F78981893409F067C05FC061E0F2
:1040900070E08BE60E941F1EF80180818093D80596
:1040A0000E948D0D53C061E070E08CE60E941F1EDF
:1040B000F0E2EF16F10461F487E6898380E2F8010B
:1040C000DE01129601900D928A95E1F761E203C03C
:1040D00087E4898361E0CE0101960E941E0C0E9454
:1040E0009C0B83E0809377056CE474E080E090E0C3
:1040F0000E94462980917705843079F58FE70E94E8
:10410000BA090E94CD09873441F520C061E070E012
:104110008DE60E941F1E89E1E816F104F1F4D80132
:10412000EEEBF5E08D91819385E0E73DF807D1F75F
:104130000E94D1130BC061E070E08EE60E941F1E4A
:10414000F80180818093D7050E946E0D81E006C042
:1041500061E070E08AEC0E941F1E80E00E94001E59
:104160000E943C1EA196E6E00C946A2FA0E0B0E00D
:10417000ECEBF0E20C944C2FCAECD3E014E606E032
:1041800035E0F32E44E0E42E53E0D52E62E0C62E57
:1041900086EE95E00E94232C892B09F49BC086EEC5
:1041A00095E00E94502C282F8093350440913404D0
:1041B00050E04730510560F7FA01EE52FF4F0C9482
:1041C000792F853B29F781E080933404E1CF823653
:1041D00009F07DC0C0923404DBCF80933304809318
:1041E0003204D0923404D4CF9C013327309331046D
:1041F0002093300490913204982790933204E092F7
:104200003404C6CF382F2227409130045091310416
:10421000242B352B309331042093300490913204B9
:10422000982790933204F09234042536310508F42F
:10423000AFCF61E070E08CEC0E941F1E81E00E9415
:10424000001E0E943C1E43C020912E0430912F047A
:10425000F901E653FC4F80839091320498279093A4
:104260003204C901019690932F0480932E0420916B
:104270003004309131048217930708F489CF0093FA
:10428000340486CF8091320482130BC060912E04D7
:1042900070912F044AEC53E0809133040E94431E36
:1042A0000DC062E070E08BEC0E941F1E8091330411
:1042B0000E94001E80916E050E94001EFE01812F4B
:1042C00011928A95E9F710922F0410922E04109201
:1042D00034045ECFCDB7DEB7E8E00C94682F81E000
:1042E00080936F0580916F05882349F086EE95E0F5
:1042F0000E94232C892BB1F30E94B620F3CF08959E
:10430000AAE2B0E0E6E8F1E20C944A2F0E941729F5
:104310006B017C0181E00E94C10A86EE95E00E945B
:10432000232C892B29F086EE95E00E94502CF5CFA6
:104330005E98409811E072E6B72EE9E2AE2E03E0F7
:104340000E9417296C197D098E099F09693C710526
:1043500081059105E0F11123D1F10E9417296B012C
:104360007C015D9A419A80ED97E00E94B607B98280
:10437000EAE7F5E0DE0112968A2D01900D928A950A
:10438000E1F76AE2CE0101960E941E0C5D98419809
:1043900080E090E00E94B607009377050E949C0B96
:1043A00062E370E080E090E00E944629809177050A
:1043B000843061F4009377058FE70E94BA090E9468
:1043C000CD0911E0823419F410E001C011E082E15E
:1043D0000E943C2A892BA1F411E012C05E9A409AF7
:1043E0005D9A419A86EE95E00E94502C8D309105A1
:1043F000B9F06CF40A97A1F05E9840985D984198E6
:1044000086EE95E00E94232C892B41F799CF8332C9
:10441000910579F08234910579F70E946F21ECCFF4
:1044200062EB71E086EE95E00E94FD2A0E94D61DA7
:10443000E3CF0E946116E0CF8F929F92AF92BF921E
:10444000CF92DF92EF92FF921F93CF93DF9382E19F
:104450000E943C2A892B09F089C068EC70E080E05A
:1044600090E00E94462980E090E00E94B6070E94FA
:1044700017294B015C016B017C0180ECC80E82E1C5
:10448000D81EE11CF11C0E9417296C157D058E05B4
:104490009F0530F482E10E943C2A892BA1F364C07D
:1044A00082E10E943C2A892B09F05EC080ED97E0F2
:1044B0000E94B6070E9417296B017C01D0E0C1E081
:1044C00088E4880E86E2981EA11CB11C11E082E1EE
:1044D0000E943C2A892B21F58C149D04AE04BF0454
:1044E00030F480ED97E00E94B607D1E0F0CF0E9453
:1044F00017296C197D098E099F09693C7105810591
:10450000910528F30E9417296B017C01C12719F03E
:1045100080ED97E002C080E090E00E94B607D7CF20
:1045200080E090E00E94B607DD23B9F08091D705C6
:1045300090E0019665E070E00E94ED2E8093D70533
:104540000E946E0D0E94EC130E948D0D64EF71E0CD
:1045500080E090E00E94462909C080E00E94DF06CA
:104560000E9405120E94840D0E948021DF91CF914C
:104570001F91FF90EF90DF90CF90BF90AF909F90F2
:104580008F900895CF92DF92EF92FF9280E00E9489
:104590001D080E94F40761E086E00E94D02961E0D6
:1045A00085E00E94D02961E08EE00E94D02961E080
:1045B0008FE00E94D02960E082E10E94D02960E073
:1045C00088E00E94D02961E088E00E94092A0E94C8
:1045D0009F0740E052EC61E070E086EE95E00E94BB
:1045E0006B2D0E94EC130E948D0D0E94D1138FEF52
:1045F0008093AA040E94090878940E9417296B01ED
:104600007C018091AA048F3F59F40E9417296C19EC
:104610007D098E099F09603D77408105910588F3EA
:1046200080ED97E00E94B60761E082E10E94092ACE
:104630005E9A409A86EE95E00E94232C892B29F001
:1046400086EE95E00E94502CF5CF6DEF72E086EE7D
:1046500095E00E94DE2A88E893E00E94730C64E1F2
:1046600073E086EE95E00E94DE2A4AE050E065E0C5
:1046700070E086EE95E00E94AE2B62E370E080E091
:1046800090E00E94462986EE95E00E94232C049734
:104690000CF186EE95E00E94502C82349105D1F405
:1046A00086EE95E00E94502C8E34910599F486EEAA
:1046B00095E00E94502C8434910561F486EE95E0DB
:1046C0000E94502C819731F480E090E00E94B60760
:1046D0000E94802140917B0550917C0560917D0571
:1046E00070917E05DB01CA010197A109B109049708
:1046F000A105B10590F44093A904433051F42EE292
:1047000040EA56E861E070E086EE95E00E94EC2D0C
:1047100008C040E052EC61E070E086EE95E00E9457
:104720006B2D0E941C225E98409880E090E00E94D1
:10473000B6070E94D1131092C9048091C30583FF6C
:1047400011C080918F05882351F0809196058823B0
:1047500031F080919D05882311F087E001C085E04C
:104760008093C90480E00E94C10A8091CA040E941B
:10477000F5090E949C0B10923F0410923E04109287
:104780003D04F12C8091D8058F15B0F062E370E004
:1047900080E090E00E94462980ED97E00E94B607F5
:1047A00062E370E080E090E00E94462980E090E0C3
:1047B0000E94B607F394E6CF8091A20584FF08C05B
:1047C000982F987181E0983109F080E00E94C11122
:1047D0008FE00E941D08FF90EF90DF90CF9008952A
:1047E000EF92FF920F931F93CF93DF938C016EE7AD
:1047F00070E086EE95E00E945906E801F12CF0E2A7
:10480000EF2E8E0188818D57823048F46DE770E07D
:1048100086EE95E00E94590688818E258883219630
:10482000F801608186EE95E00E947D2CF394F9E01A
:10483000FF12E7CF6EE770E086EE95E00E94590622
:10484000CDB7DEB7E6E00C946A2FA9E0B0E0EBE26A
:10485000F4E20C94522F9091CB0491110EC09EEF74
:1048600099838A836B8350E0559547954C832D83BC
:10487000198618861F821E822EC04091D004842F74
:1048800090E0B4E095958795BA95E1F7242F2F70C5
:1048900030E08217930719F18DEF89831B82FE01A7
:1048A000349650E0842F90E0A4E095958795AA95E2
:1048B000E1F7242F2F7030E08217930749F0DC01D5
:1048C000AF52BB4F8C918193405F5F5F563051F781
:1048D0004093D0045A83CE0101960E94F023809128
:1048E000CB0490E0019666E070E00E94ED2E80938C
:1048F000CB042996E2E00C946E2FA0E0B0E0E3E850
:10490000F4E20C944B2F6C016EE770E086EE95E0BC
:104910000E9459068601E12CF12CC0E0D0E030E283
:10492000B32EF801608183E8860F823078F46DE75A
:1049300070E086EE95E00E945906F80160816B25D3
:1049400070E086EE95E00E94590604C086EE95E080
:104950000E947D2CE114F10459F0F80180819E0140
:10496000280F311DC901C92FDD27C80FD91FDD2729
:104970003FEFE31AF30A89E0E816F10459F028E062
:10498000E216F10421F48C2F8095F60180870F5FE9
:104990001F4FC7CFCDB7DEB7E9E00C94672FA9E072
:1049A000B0E0E5EDF4E20C94522FE82F362F809121
:1049B000CB0490E0019664E270E00E94ED2E8093BB
:1049C000CB0458E9598350E15A83813089F048F08B
:1049D0008230B9F08330D9F48B8381EF8C833D83AF
:1049E00019C085E08B8381EF8C832F5F2D8312C0EC
:1049F0008B8381EF8C8384E6489FA00111245D8323
:104A000009C084E08B8381EF8C83ED8303C00E9417
:104A1000FE1104C0CE0101960E947D242996E2E099
:104A20000C946E2FA2E0B0E0E8E1F5E20C94472F81
:104A3000182F762E2A8349830E9423296B017C013B
:104A40008091E1048090CC049090CD04A090CE049D
:104A5000B090CF042A8149818823C1F0D701C601D3
:104A600088199909AA09BB094C015D0191EE8916C3
:104A70009EE29906A104B10420F1241708F4422F04
:104A8000202F672D812F0E94CF2413C0D701C6018C
:104A900088199909AA09BB094C015D0191E389169E
:104AA00095E79906A104B10460F0672D812F0E945B
:104AB0002524C092CC04D092CD04E092CE04F09292
:104AC000CF042296EDE00C94632FA2E2B0E0EBE677
:104AD000F5E20C94482F8CE00E94DC0981110FC094
:104AE0006CE173E086EE95E00E940F2B5E9A409A8F
:104AF00080E00E94C10A0E949C0B5E98409886EE5E
:104B000095E00E94232C892B01F186EE95E00E940E
:104B1000502C9091A904992319F00E94FF13EFCF14
:104B200040913E0450E09A012F5F3F4F2F71332791
:104B300060913F0470E02617370709F3FA01E75B3D
:104B4000FB4F808320933E04DACF80917705843039
:104B500009F086C00E942329611571058105910520
:104B600049F06093BB047093BC048093BD049093A0
:104B7000BE040CC081E090E0A0E0B0E08093BB04F4
:104B80009093BC04A093BD04B093BE048091AD0487
:104B90009091AE0481609093AE048093AD0483E065
:104BA000809377058FE70E94BA0909E614E00E9416
:104BB000CD09F80181938F01F4E002371F07B9F79F
:104BC0002091720480916904982F922796FF3BC030
:104BD00090E4922790937204982F98739833F1F48D
:104BE00010E0212F30E080916904877090E08217F7
:104BF00093074CF11F5F2091A205812F90E0FC01EB
:104C0000E759FB4F24FF04C080810E94E011E9CFE7
:104C1000608186EE95E00E947D2CE3CF8F7399F43E
:104C200080916A048093B60480916B048093B404ED
:104C300080916C048093B30480916F0490E0909312
:104C4000AC048093AB0480913D04813019F482E080
:104C500080933D0480913D04833011F410923D0413
:104C60000E9423296B017C018091AF049091B004D4
:104C7000A091B104B091B2040097A105B105C9F0AB
:104C8000A7019601281B390B4A0B5B0BDA01C901FE
:104C9000883B9B40A105B10560F00E940B0A809300
:104CA000B5041092AF041092B0041092B1041092A7
:104CB000B2048091BF049091C004A091C104B0914E
:104CC000C20446015701881A990AAA0ABB0A8AE750
:104CD00095E00E94370886169706A806B90608F4DC
:104CE000A9C0C092BF04D092C004E092C104F09267
:104CF000C2040E9457068091AA048830A0F08091D7
:104D0000C3059091C405A091C505B091C6055CE1AD
:104D1000B695A795979587955A95D1F7892B8A2BA4
:104D20008B2B09F0AEC18091AA048F5F8093AA04F7
:104D30008091BB049091BC04A091BD04B091BE04CD
:104D40000097A105B105F1F0C81AD90AEA0AFB0AD1
:104D50008AE795E00E9437086C157D058E059F0552
:104D600008F014C18091C30584FD04C080ED97E074
:104D70000E94B6071092BB041092BC041092BD04AE
:104D80001092BE0490917204907C909372045091A2
:104D90003E0480913F0420913D04581709F413C14B
:104DA000223009F010C1905890937204E091A2054E
:104DB000E770F0E0E658FC4F6081693008F0EBC026
:104DC000615040E04613E9C080933F0487E3840FBD
:104DD00090917204892B809372044093400483E085
:104DE00080933D045D9A419A809187059091C90412
:104DF000911138C10E94BC0A8091CA040E94F50931
:104E0000E091A205E770F0E0E658FC4F608182E790
:104E100094E00E94D70BE091CA04EF5FE093CA04CC
:104E2000E83109F42BC1F0E0E658FA4F8785882372
:104E300009F424C10E94460C813069F58091A205D5
:104E4000887149F18091AD049091AE04880F991F4B
:104E50009093AE048093AD0483E0809377050E9425
:104E60009C0B0E9423296093AF047093B00480933D
:104E7000B1049093B204672B682B692B61F481E035
:104E800090E0A0E0B0E08093AF049093B004A093D2
:104E9000B104B093B2048091A20584FF2BC080912D
:104EA000BB049091BC04A091BD04B091BE04892BB9
:104EB0008A2B8B2BF9F08091AD049091AE048E7FFC
:104EC0000E946D09182F6091AB048091B6040E9476
:104ED000F513482F612F8091B50449A30E94F51363
:104EE0000091D805282F49A16091B3048091B404A2
:104EF0000E9412255D9841988091C7048130C1F0CD
:104F000018F08230B1F1CBC082E10E943C2A892B9B
:104F100009F0C5C081E08093C7040E9417296093FF
:104F2000C3047093C4048093C5049093C604B7C0AF
:104F300082E10E943C2A892B31F50E941729C090FA
:104F4000C304D090C404E090C504F090C6046C196A
:104F50007D098E099F09693E73408105910508F41A
:104F60009EC082E08093C70480ED97E00E94B60760
:104F700096C082E10E943C2A892B09F490C080E00F
:104F800090E00E94B6071092C70489C080E090E0CC
:104F90000E94B607F7CE68E014CF851709F414CF46
:104FA0004F5F242F30E090E0F901EE58FB4FDC0119
:104FB000A75BBB4F7C917083F901E05CFB4F708372
:104FC00001968F71FFCE2430B1F42091400481E42A
:104FD00094E0A3E7B4E0FC013E2F381B321718F42D
:104FE00031913D93F9CF87E3820F90917204892B21
:104FF00080937204F4CE8091C704823059F491609A
:10500000909372045E9A409A8E010F5F1F4FF12CAD
:10501000B80111C05E98409880913D04811103C091
:1050200081E080933D0480913D04833069F784E002
:1050300080933D04E9CF8F2D69A37AA30E941E16A9
:10504000F801819391938F01F39469A17AA1F0E122
:10505000FF12F1CF8091A20543E754E087700E94D0
:10506000BC08C0CE882309F4C5CE2091C80431E025
:10507000320F3093C8042913BDCE0DC01092CA045C
:10508000D9CE8091AA04883011F45E9A409A89E0C2
:105090008093AA04CFCE1092C8048150ABCEA296C2
:1050A000ECE00C94642F8230E8F4E82FF0E0EE0F8F
:1050B000FF1FE752FA4F71836083813041F0809186
:1050C00069008C7F842B80936900E89A0895809111
:1050D0006900440F551F440F551F837F842B809315
:1050E0006900E99A08951F920F920FB60F9211244A
:1050F0002F933F934F935F936F937F938F939F93E0
:10510000AF93BF93EF93FF938091D9059091DA0508
:10511000892B29F0E091D905F091DA050995FF91E5
:10512000EF91BF91AF919F918F917F916F915F911F
:105130004F913F912F910F900FBE0F901F90189598
:105140001F920F920FB60F9211242F933F934F93FC
:105150005F936F937F938F939F93AF93BF93EF93DF
:10516000FF938091DB059091DC05892B29F0E0917C
:10517000DB05F091DC050995FF91EF91BF91AF91AF
:105180009F918F917F916F915F914F913F912F915F
:105190000F900FBE0F901F9018951F920F920FB691
:1051A0000F9211242F933F938F939F93AF93BF93AD
:1051B0008091DE059091DF05A091E005B091E105B9
:1051C0003091DD0523E0230F2D3720F40196A11D3A
:1051D000B11D05C026E8230F0296A11DB11D209325
:1051E000DD058093DE059093DF05A093E005B09385
:1051F000E1058091E2059091E305A091E405B0916D
:10520000E5050196A11DB11D8093E2059093E3058C
:10521000A093E405B093E505BF91AF919F918F9165
:105220003F912F910F900FBE0F901F9018952FB7A1
:10523000F8946091DE057091DF058091E005909112
:10524000E1052FBF08953FB7F8948091E205909152
:10525000E305A091E405B091E50526B5A89B05C03E
:105260002F3F19F00196A11DB11D3FBF6627782F72
:10527000892F9A2F620F711D811D911D42E0660FCB
:10528000771F881F991F4A95D1F70895CF92DF9213
:10529000EF92FF92CF93DF936B017C010E94232951
:1052A000EB01C114D104E104F10479F00E94232937
:1052B0006C1B7D0B683E7340A0F381E0C81AD108D7
:1052C000E108F108C851DC4FECCFDF91CF91FF909E
:1052D000EF90DF90CF900895789484B5826084BD7C
:1052E00084B5816084BD85B5826085BD85B58160EA
:1052F00085BDEEE6F0E0808181608083E1E8F0E04A
:105300001082808182608083808181608083E0E878
:10531000F0E0808181608083E1EBF0E08081846057
:105320008083E0EBF0E0808181608083EAE7F0E059
:1053300080818460808380818260808380818160BD
:1053400080838081806880831092C10008958330BB
:1053500081F028F4813099F08230A1F008958630F0
:10536000A9F08730B9F08430D1F4809180008F7D2E
:1053700003C0809180008F7780938000089584B56A
:105380008F7702C084B58F7D84BD08958091B00071
:105390008F7703C08091B0008F7D8093B000089517
:1053A000CF93DF9390E0FC01ED50F44F2491FC018A
:1053B000E95FF34F8491882349F190E0880F991FAA
:1053C000FC01E15DF34FA591B4918B5D934FFC011E
:1053D000C591D4919FB7611108C0F8948C91209524
:1053E00082238C93888182230AC0623051F4F8941E
:1053F0008C91322F309583238C938881822B8883E4
:1054000004C0F8948C91822B8C939FBFDF91CF9135
:105410000895A1E0B0E0EFE0FAE20C94502F282FBD
:1054200030E0F901E152F44F8491F901ED50F44F6D
:105430001491F901E95FF34F04910023C9F0882327
:1054400021F069830E94A7296981E02FF0E0EE0F27
:10545000FF1FEB5DF34FA591B4919FB7F8948C912A
:10546000611103C01095812301C0812B8C939FBFD4
:105470002196E4E00C946C2FCF93DF93282F30E03B
:10548000F901E152F44F8491F901ED50F44FD491B8
:10549000F901E95FF34FC491CC2391F081110E948F
:1054A000A729EC2FF0E0EE0FFF1FE55EF34FA5916B
:1054B000B4912C912D2381E090E021F480E002C092
:1054C00080E090E0DF91CF9108958E3008F08E500B
:1054D000877020919D0190E4299F90011124822BD7
:1054E00080937C0080917A00806480937A00809120
:1054F0007A0086FDFCCF809178002091790090E0C1
:10550000922B0895A0E0B0E0E8E8FAE20C944C2F6A
:105510006C017A01EB01E60EF71E00E010E0CE15FB
:10552000DF0561F06991D601ED91FC910190F08168
:10553000E02DC6010995080F191FF1CFC801CDB79D
:10554000DEB7E8E00C94682F6115710589F0DB0186
:105550000D900020E9F7AD0141505109461B570B52
:10556000DC01ED91FC910280F381E02D0995089515
:1055700080E090E00895EF92FF920F931F93CF93F6
:10558000DF938C01FB01C0E0D0E064917F018FEFDD
:10559000E81AF80A662361F0D801ED91FC910190B8
:1055A000F081E02DC8010995C80FD91FF701EDCF93
:1055B000CE01CDB7DEB7E6E00C946A2F0E94A42A94
:1055C0000895DC01ED91FC910190F081E02D0995A9
:1055D00008950F931F93CF93DF93EC016DE00E942A
:1055E000E12A8C016AE0CE010E94E12A800F911F1E
:1055F000DF91CF911F910F9108950F931F93CF9338
:10560000DF93EC010E94BB2A8C01CE010E94E92AA3
:10561000800F911FDF91CF911F910F9108950F93EC
:105620001F93CF93DF93EC010E94A42A8C01CE013B
:105630000E94E92A800F911FDF91CF911F910F9156
:1056400008950F931F93CF93DF93EC010E94E12AFB
:105650008C01CE010E94E92A800F911FDF91CF912A
:105660001F910F910895A1E2B0E0E9E3FBE20C94F1
:10567000482F7C01C42EE52FCB01D22E19A221E0A8
:105680002D1510F02AE0D22E8E010F5D1F4F8D2CAC
:10569000912CA12CB12C6C2D7E2FA50194010E9480
:1056A000012F8C2DD29E80191124015011098A30AE
:1056B00010F4805D01C0895CF801808321153105FB
:1056C0004105510521F0C22EE32FCA01E4CFB801F4
:1056D000C7010E94A42AA196ECE00C94642FA0E0DC
:1056E000B0E0E5E7FBE20C944C2FEC016A017B0192
:1056F0002115310541F4E881F9810190F081E02D17
:10570000642F09951DC02A303105A9F477FF12C016
:105710006DE20E94E12A8C0144275527BA014C19F9
:105720005D096E097F092AE0CE010E94332B800FAC
:10573000911F06C02AE0B701A601CE010E94332BBB
:10574000CDB7DEB7E8E00C94682F9A01AB0166276D
:1057500057FD6095762F0E946F2B08950F931F932E
:10576000CF93DF93EC019A01AB01662757FD60955B
:10577000762F0E946F2B8C01CE010E94E92A800FA8
:10578000911FDF91CF911F910F9108952115310540
:1057900049F4DC01ED91FC910190F081E02D642F42
:1057A000099508950E94332B08959A01462F50E0E1
:1057B00060E070E00E94C62B08959A01AB0160E0A2
:1057C00070E00E94C62B08950F931F93CF93DF9331
:1057D000EC010E94C62B8C01CE010E94E92A800FA9
:1057E000911FDF91CF911F910F9108950F931F93F8
:1057F000CF93DF93EC019A01AB0160E070E00E946F
:10580000C62B8C01CE010E94E92A800F911FDF91E7
:10581000CF911F910F9108950F931F93CF93DF9313
:10582000EC019A01462F50E060E070E00E94C62B28
:105830008C01CE010E94E92A800F911FDF91CF9148
:105840001F910F910895FC0124853585F901E05CD5
:10585000FF4F80819181F901EE5BFF4F2081318103
:10586000821B930B8F7399270895FC01848595857E
:10587000FC01E05CFF4F40815181FC01EE5BFF4F7A
:10588000208131814217530741F00190F081E02DD2
:10589000E80FF91F808190E008958FEF9FEF089542
:1058A000FC0184859585FC01E05CFF4F40815181BE
:1058B000FC01EE5BFF4F208131814217530779F0E5
:1058C000A081B181A80FB91F8C91208131812F5FF8
:1058D0003F4F2F7333273183208390E008958FEF5C
:1058E0009FEF0895FC0181A1882329F0A489B5893F
:1058F0008C9186FFFBCF11A20895CF93DF93FC011B
:1059000026853785D901A05CBF4F8D919C91119759
:1059100001968F739927E901CE5BDF4F488159814A
:1059200084179507D9F30D90BC91A02DA20FB31F3A
:105930006C93A685B785A05CBF4F11969C938E9300
:10594000A689B7892C9181E090E0078C02C0880F6E
:10595000991F0A94E2F7282B2C9381E081A30488F5
:10596000F589E02D80818064808381E090E0DF9183
:10597000CF91089508951F920F920FB60F921124A0
:105980002F933F934F938F939F93EF93FF93809128
:10599000C00082FD1CC04091C60080918C06909191
:1059A0008D0601968F73992720918E0630918F0670
:1059B0008217930771F0E0918C06F0918D06E45BFD
:1059C000F94F408390938D0680938C0602C080919E
:1059D000C600FF91EF919F918F914F913F912F9131
:1059E0000F900FBE0F901F90189586EE95E00E94C5
:1059F000232C892B11F00E94BA2C08951F920F922C
:105A00000FB60F9211242F933F938F939F93EF9391
:105A1000FF93209148063091490680914A06909163
:105A20004B062817390731F48091C1008F7D809390
:105A3000C10014C0E0914A06F0914B06E85FF94FAF
:105A4000208180914A0690914B0601968F73992789
:105A500090934B0680934A062093C600FF91EF91E6
:105A60009F918F913F912F910F900FBE0F901F909C
:105A70001895A0E0B0E0EFE3FDE20C94482FFC01A4
:105A80001382128288EE93E0A0E0B0E084839583D5
:105A9000A683B7838CEB93E09183808375876487BB
:105AA00057874687318B208B138B028BF58AE48ACC
:105AB000D78AC68AB18EA08E938E828E8F85848F70
:105AC0008889858F8989868F8A89878F8B8980A32A
:105AD000ECE00C94642FCF92DF92EF92FF92CF9381
:105AE000DF93EC016A017B01411581EE58076105E6
:105AF0007105F9F0EC89FD8981E090E008A002C011
:105B0000880F991F0A94E2F7808360E079E08DE3C3
:105B100090E0A70196010E94012F2150310941090F
:105B200051095695479537952795211580E13807F6
:105B300098F0EC89FD89108260E874E88EE190E0CD
:105B4000A70196010E94012F2150310941095109F5
:105B50005695479537952795E889F9893083EA89DD
:105B6000FB89208319A2EE89FF89408181E090E0C2
:105B70009C010C8C02C0220F331F0A94E2F7422BC7
:105B80004083EE89FF8940819C010D8C02C0220F69
:105B9000331F0A94E2F7422B4083EE89FF8940814C
:105BA0009C010E8C02C0220F331F0A94E2F7422B95
:105BB0004083EE89FF8920810F8C02C0880F991FD6
:105BC0000A94E2F7809582238083DF91CF91FF9042
:105BD000EF90DF90CF900895BF92CF92DF92EF9237
:105BE000FF92CF93DF93EC016A017B01B22E411546
:105BF00081EE580761057105F9F0EC89FD8981E0B6
:105C000090E008A002C0880F991F0A94E2F78083F1
:105C100060E079E08DE390E0A70196010E94012FFA
:105C200021503109410951095695479537952795D6
:105C3000211580E1380798F0EC89FD89108260E831
:105C400074E88EE190E0A70196010E94012F215097
:105C50003109410951095695479537952795E889A6
:105C6000F9893083EA89FB892083E88DF98DB08238
:105C7000EE89FF89408181E090E09C010C8C02C09C
:105C8000220F331F0A94E2F7422B4083EE89FF89EB
:105C900040819C010D8C02C0220F331F0A94E2F751
:105CA000422B4083EE89FF8940819C010E8C02C00B
:105CB000220F331F0A94E2F7422B4083EE89FF89BB
:105CC00020810F8C02C0880F991F0A94E2F78095FB
:105CD00082238083DF91CF91FF90EF90DF90CF9070
:105CE000BF9008958F929F92AF92BF92CF92DF9212
:105CF000EF92FF920F931F9381E08F9385E08F9334
:105D000087E08F9383E08F9384E08F93E6EC8E2E71
:105D1000912CF2ECAF2EB12CA1ECCA2ED12CB0EC10
:105D2000EB2EF12C04EC10E025EC30E048E056E0DE
:105D30006CE476E086EE95E00E94392D0F900F908E
:105D40000F900F900F901F910F91FF90EF90DF90A9
:105D5000CF90BF90AF909F908F9008950E946C2934
:105D60000E94C222C5EFDCE20E9465252097E1F384
:105D70000E94F52CF9CFA29FB001B39FC001A39F51
:105D8000700D811D1124911DB29F700D811D112474
:105D9000911D08950E94BB2EA59F900DB49F900D5C
:105DA000A49F800D911D11240895B7FF0C94CA2E55
:105DB0000E94CA2E821B930B0895DB018F939F9341
:105DC0000E94CA2EBF91AF91A29F800D911DA39FEB
:105DD000900DB29F900D1124089597FB072E16F495
:105DE000009407D077FD09D00E947F2F07FC05D0D3
:105DF0003EF4909581959F4F0895709561957F4FE2
:105E00000895A1E21A2EAA1BBB1BFD010DC0AA1FFB
:105E1000BB1FEE1FFF1FA217B307E407F50720F013
:105E2000A21BB30BE40BF50B661F771F881F991F8E
:105E30001A9469F760957095809590959B01AC01D7
:105E4000BD01CF010895052E97FB1EF400940E941A
:105E50003A2F57FD07D00E94012F07FC03D04EF4C4
:105E60000C943A2F50954095309521953F4F4F4FC8
:105E70005F4F089590958095709561957F4F8F4FF6
:105E80009F4F08952F923F924F925F926F927F9211
:105E90008F929F92AF92BF92CF92DF92EF92FF923A
:105EA0000F931F93CF93DF93CDB7DEB7CA1BDB0BE6
:105EB0000FB6F894DEBF0FBECDBF09942A8839888B
:105EC00048885F846E847D848C849B84AA84B98492
:105ED000C884DF80EE80FD800C811B81AA81B9819E
:105EE000CE0FD11D0FB6F894DEBF0FBECDBFED01B2
:105EF0000895EE0FFF1F0590F491E02D0994AA1B61
:105F0000BB1B51E107C0AA1FBB1FA617B70710F0A4
:105F1000A61BB70B881F991F5A95A9F780959095D6
:105F2000BC01CD0108958F929F92AF92BF92CF9204
:105F3000DF92EF92FF92CF93DF93EC01688179813A
:105F40008A819B81611571058105910521F464E2C7
:105F500079ED8BE597E02DE133EF41E050E00E94D1
:105F6000232F49015A019B01AC01A7EAB1E40E9429
:105F7000CA2E6B017C01ACEEB4EFA50194010E9426
:105F8000D82EC60ED71EE81EF91EF7FE06C081E009
:105F9000C81AD108E10880E8F80AC882D982EA82E2
:105FA000FB82C701B6019F77DF91CF91FF90EF9001
:105FB000DF90CF90BF90AF909F908F9008950E94F8
:105FC000932F089586E091E00E94932F08956093A7
:105FD00006017093070180930801909309010895C9
:105FE0002F923F925F926F927F928F929F92AF9289
:105FF000BF92CF92DF92EF92FF920F931F93CF93B6
:10600000DF938B01EA016115710521F0DB018C93AF
:1060100011969C93209739F09E012250310923322A
:10602000310508F0D8C07C016701BFEFCB1ADB0A4D
:106030005601F7016080862D90E00E942231892B65
:1060400011F07601F1CFFDE26F120AC0570182E034
:10605000A80EB11CD70111966C90772473940BC0D5
:10606000BBE26B1207C05701E2E0AE0EB11CD701D4
:1060700011966C90712CCE018F7E892B89F4B0E340
:106080006B1237C0F50180818F7D8835D1F4618036
:10609000F2E0AF0EB11C872D8260782EC0E1D0E017
:1060A000CA30D10551F1C031D10521F0C830D10538
:1060B00099F409C0CC24CA94DC2CEC2CAFE0FA2E65
:1060C00022C0209769F7C8E0D0E0CC24CA94DC2C29
:1060D000EC2CFFE1FF2E17C06FEF7FEFCB019E018D
:1060E000442737FD4095542F0E94012F69017A0102
:1060F0000AC02097A9F6CAE0D0E0E9E9CE2EDC2C50
:10610000EC2CE9E1FE2EF50160E020E030E0A90191
:106110004E01AA2497FCA094BA2C1F0170ED572EB3
:10612000560CA9E0A51570F48FEB860D8A3118F492
:1061300099EC592E06C08FE9860D8A3148F589EA17
:10614000582E560C852D90E08C179D070CF56F3F4F
:10615000D9F0C216D306E406F50698F0C501B401DD
:106160000E94DD2E9B01AC01852D90E0A0E0B0E007
:10617000280F391F4A1F5B1F281739074A075B077B
:1061800010F46FEF01C061E03196D1016C90C5CF82
:106190000115110551F0662311F0319703C071FE0E
:1061A00004C03297D801ED93FC9370FE07C0509560
:1061B0004095309521953F4F4F4F5F4F67FF10C07F
:1061C00082E290E090939106809390066FEF7FEFCC
:1061D0008FEF9FEF07C060E070E080E090E002C0CA
:1061E000B901CA01DF91CF911F910F91FF90EF90FC
:1061F000DF90CF90BF90AF909F908F907F906F90E7
:106200005F903F902F900895FC0188279927E8948C
:1062100021912032E9F3293010F02E30C8F32B32CF
:1062200041F02D3239F4689404C00E945631820F37
:10623000911D219120532A30C0F31EF49095819531
:106240009F4F0895911150C0803219F089508550A8
:10625000D0F7089548EC53E00E942F310895FA01D9
:10626000A191B081009719F41097E1F0CD01DC0104
:10627000CD010D90002011F4C00113C0FB0121914C
:10628000222319F02015D9F7F3CFFB012191201516
:1062900019F41E92119606C02223C1F70D9000201A
:1062A000A1F7D001FA01A193B08308957AE0979FF6
:1062B000902D879F802D910D11240895F999FECF7F
:1062C00092BD81BDF89A992780B50895262FF99936
:1062D000FECF1FBA92BD81BD20BD0FB6F894FA9AC9
:1062E000F99A0FBE01960895992788270895F89482
:0262F000FFCFDE
:1062F20000009206200001000000FF0002000200E0
:10630200020002000200020002000200020002007B
:1063120002000200020002000200028025000005C5
:10632200400AA1204EA50020244EA52C2330C012E5
:1063320000001A400AA1204EA5001B1E27522C2342
:10634200308025000005400AA1204EA50020244EE1
:10635200A52C2330004B000006400AD0009D4900C6
:106362007B289D492C233000E1000005400A4501AD
:10637200D7DC03B81E0EBF00232E48E801008A4076
:106382000A6001555502AD1E20000023C801545871
:106392002074696D656F75742100596573004E6FC5
:1063A200002C00386368004E2F41002C205B005DFA
:1063B2002028002900486F70206368616E6E656C4A
:1063C200200020402000456E746572696E6720616E
:1063D20064617074697665206368616E6E656C20B5
:1063E20073656C656374696F6E2C207069636B6989
:1063F2006E673A007363616E6E6572206D6F6465DD
:10640200004E4F5420454E41424C45440053656E68
:1064120064696E672073657474696E677320746F44
:106422002052580A00526573657474696E6720734E
:10643200657474696E6773206F6E2052580A00414A
:10644200626F727465642065646974730A00696EB0
:1064520076616C69642073656C656374696F6E0044
:106462000D0A496E76616C696420696E70757420DC
:106472002D2064697363617264656421070053654A
:106482007474696E677320736176656420746F201B
:10649200454550524F4D0A005265766572746564E7
:1064A2002073657474696E67732066726F6D204520
:1064B2004550524F4D0A004C6F616465642066611D
:1064C20063746F72792064656661756C74730A0017
:1064D2004B657920616E64206368616E6E656C73D2
:1064E2002072616E646F6D697A65640A004F70652F
:1064F2006E4C52536E6720545820737461727469E3
:106502006E672000206F6E20485720006D6F647503
:106512006C65206C6F636B65643F00342B3400380C
:1065220000382B340031320031322B340031360046
:1065320050504D0052535349005344410053434C71
:1065420000525844005458440041494E004C4245C0
:1065520045500053504B54524D0053425553005333
:10656200554D44004C4C494E440000070B0C101191
:106572001500B7012B032F033103350338033D0305
:10658200B7014003440349034D0351035503590323
:106592005D0363036A036F0374038D028D028D0230
:1065A2008D02160A13223129000000007D2C822A56
:0865B200232C502C352C722C17
:00000001FF
